:100000000C9434000C9433020C9457020C9451005D
:100010000C9451000C9451000C9451000C9451001C
:100020000C9451000C9451000C9451000C9451000C
:100030000C9451000C9451000C9451000C945100FC
:100040000C9451000C9451000C9451000C945100EC
:100050000C9451000C9451000C9451000C945100DC
:100060000C9451000C94510011241FBECFEFD8E026
:10007000DEBFCDBF11E0A0E0B1E0EAE2F9E002C0EE
:1000800005900D92AE38B107D9F721E0AEE8B1E0A6
:1000900001C01D92A939B207E1F70E9423040C9414
:1000A00093040C9400003D9A3C9A3B9A3A9A399AF0
:1000B000389A0895459888230CF4459A449886FD0B
:1000C000449A439885FD439A429884FD429A419A06
:1000D0008AEB8A95F1F700C041988AEB8A95F1F78F
:1000E00000C00895CF93C82F409A41980E945A00AB
:1000F0008C2F8295807F0E945A00CF9108950F9394
:100100001F93CF93DF9300D0CDB7DEB78C011A8257
:100110001982E981FA81E80FF91F80818823B1F003
:10012000E981FA81E00FF11F80810E9472008981CC
:100130009A8101969A83898380EF8A95F1F7E98104
:10014000FA81E00FF11F80818111EACF0F900F90AB
:10015000DF91CF911F910F910895CF93C82F4098B1
:1001600041980E945A008C2F8295807F0E945A00ED
:10017000CF9108952FEF80E792E02150804090408A
:10018000E1F700C000004098419880E30E945A00C7
:100190008FE39CE90197F1F700C0000080E30E9423
:1001A0005A0087E592E00197F1F700C0000080E374
:1001B0000E945A0087E592E00197F1F700C0000025
:1001C00088E20E945A0090EF9A95F1F788E20E9427
:1001D000AD0020EF2A95F1F788E00E94AD0080EF96
:1001E0008A95F1F781E00E94AD008FE79EE30197C9
:1001F000F1F700C0000086E00E94AD0090EF9A95F4
:10020000F1F78CE00E94AD0020EF2A95F1F70895F8
:1002100041E0682F80E10E943A04089541E0682F90
:1002200080E00E943A04089542E0682F81E10E9434
:100230003A04089542E0682F82E10E943A0408954A
:1002400080E80E94AD0081E091E00E947F0080EC98
:100250000E94AD0082E191E00E947F000895E9E6EE
:10026000F0E08081856080838DB383608DBB78945E
:1002700008958AB1827F8AB908950E942F010E9451
:1002800039010E9453000E94BA000E9456040E9445
:10029000200180E00E94140180E00E940E0180E0B5
:1002A0000E941A0180E00E9408010895CF93DF9315
:1002B00000D0CDB7DEB71A82198289B182FB8827B8
:1002C00080F98093950189B183FB882780F9809319
:1002D00094018BE291E00197F1F700C0000080915A
:1002E0009501811112C080919301882371F0809152
:1002F0009401882329F081E090E09A83898307C0E4
:100300008FEF9FEF9A83898302C01A8219828091AE
:1003100095018093930189819A810F900F90DF91CD
:10032000CF91089510928E0180910001833079F170
:1003300018F4823041F00895843009F44CC08530BF
:1003400009F46DC008950E9456018F3F2FEF920768
:1003500019F0019761F016C080919201823018F473
:10036000109292010FC08350809392010BC0809134
:1003700092018A3F20F08FEF8093920103C08D5F3E
:1003800080939201809192010E94080108950E9439
:1003900056018F3F2FEF920719F0019761F016C0B9
:1003A00080919101823018F4109291010FC0815018
:1003B000809391010BC0809191018E3F20F08FEFCF
:1003C0008093910103C08F5F80939101809191018F
:1003D0000E940E0108950E9456018F3F2FEF920751
:1003E00019F0019761F016C080918F01823018F4E6
:1003F00010928F010FC0835080938F010BC08091AA
:100400008F018E3F20F08FEF80938F0103C08D5FAF
:1004100080938F0180918F010E94140108950E94A2
:1004200056018F3F2FEF920719F0019761F016C028
:1004300080919001823018F4109290010FC0835087
:10044000809390010BC0809190018E3F20F08FEF40
:100450008093900103C08D5F809390018091900103
:100460000E941A0108951F920F920FB60F92112445
:100470002F933F934F935F936F937F938F939F93AC
:10048000AF93BF93EF93FF930E949201FF91EF917F
:10049000BF91AF919F918F917F916F915F914F919C
:1004A0003F912F910F900FBE0F901F9018951F92A4
:1004B0000F920FB60F9211242F933F934F935F9398
:1004C0006F937F938F939F93AF93BF93EF93FF931C
:1004D0000E949201FF91EF91BF91AF919F918F91F7
:1004E0007F916F915F914F913F912F910F900FBE30
:1004F0000F901F9018952DEC829F912D11249695A9
:1005000096959695492F440F342F330F330F340FA0
:10051000482F431B342F305DE6E9F1E03283929F90
:10052000212D1124269526952695220F322F330F43
:10053000330F230F921B905D918399E2899F812D48
:10054000112482958F70805D80830895CF93DF930F
:1005500080919001C4E6C89FC00111246FEF70E044
:100560000E946B04862F0E947B0280E80E94AD00EF
:1005700083E291E00E947F0080EC0E94AD0084E362
:1005800091E00E947F0080919001C89FC0011124DA
:100590009C0122503F4F243F3A4040F489EC0E9496
:1005A000AD00809198010E9472001BC0865F994047
:1005B000863A994578F488EC0E94AD00C6E9D1E00E
:1005C00089810E94720089EC0E94AD008A810E949C
:1005D000720007C087EC0E94AD0085E491E00E94A4
:1005E0007F00DF91CF910895CF93DF9380919101A8
:1005F000C4E6C89FC00111246FEF70E00E946B0435
:10060000862F0E947B0280E80E94AD0089E491E081
:100610000E947F0080EC0E94AD0084E391E00E9484
:100620007F0080919101C89FC00111249C0122503C
:100630003F4F243F3A4040F489EC0E94AD00809146
:1006400098010E9472001BC0865F9940863A9945C6
:1006500078F488EC0E94AD00C6E9D1E089810E945F
:10066000720089EC0E94AD008A810E94720007C06E
:1006700087EC0E94AD0085E491E00E947F00DF914D
:10068000CF910895CF93DF9380919201C4E6C89FE4
:10069000C00111246FEF70E00E946B04862F0E944E
:1006A0007B0280E80E94AD008AE591E00E947F0015
:1006B00080EC0E94AD008BE691E00E947F0080916B
:1006C0009201C89FC00111249C0122503F4F243F3A
:1006D0003A4040F48AEC0E94AD00809198010E945B
:1006E00072001BC0865F9940863A994578F489EC80
:1006F0000E94AD00C6E9D1E089810E9472008AECB7
:100700000E94AD008A810E94720007C088EC0E949E
:10071000AD0085E491E00E947F00DF91CF910895C4
:10072000CF93DF9380918F01C4E6C89FC00111244D
:100730006FEF70E00E946B04862F0E947B0280E8BE
:100740000E94AD008CE791E00E947F0080EC0E9447
:10075000AD0084E391E00E947F0080918F01C89FEB
:10076000C00111249C0122503F4F243F3A4040F4E5
:1007700089EC0E94AD00809198010E9472001BC01C
:10078000865F9940863A994578F488EC0E94AD00DE
:10079000C6E9D1E089810E94720089EC0E94AD0017
:1007A0008A810E94720007C087EC0E94AD0085E438
:1007B00091E00E947F00DF91CF9108951F93CF9326
:1007C000DF9315E0C1E0D4E0809100018430A9F00E
:1007D000853021F18330D1F780918E01811104C0E1
:1007E0000E94F402C0938E014899EECF10928E01C0
:1007F000489BFECFD0930001E7CF80918E018111FD
:1008000004C00E949003C0938E014899DDCF1092DE
:100810008E01489BFECF10930001D6CF80918E01B0
:10082000811104C00E94A602C0938E014899CCCFCA
:10083000489BFECF82E08093000110928E01DF91F1
:10084000CF911F9108950E943D01C1E0D3E08091B6
:100850008E01811104C00E944203C0938E01489909
:10086000F6CF10928E01489BFECFD09300010E94DC
:10087000DE03EDCF95B121E030E002C0220F331F3F
:100880004A95E2F7422F4095942395B995E09A95C1
:10089000F1F700008EBD0DB407FEFDCF6EBD0DB4A7
:1008A00007FEFDCF85B1282B25B908958EE284B9C6
:1008B00085B1866085B980E58CBD81E08DBD8FEC0A
:1008C00097E00197F1F700C0000041E06FEF80E48E
:1008D0000E943A04089597FB072E16F4009407D05F
:1008E00077FD09D00E947F0407FC05D03EF4909567
:1008F00081959F4F0895709561957F4F0895AA1B2C
:10090000BB1B51E107C0AA1FBB1FA617B70710F0FA
:10091000A61BB70B881F991F5A95A9F7809590952C
:0A092000BC01CD010895F894FFCF4B
:10092A00024772656574696E6773203A2920202030
:10093A002000416D706C6966696365206973204F98
:10094A004E20003C2044656C61792054696D652015
:10095A0020203E003C56616C75653A2020205B25BC
:10096A005D20203E00313030003C204761696E2016
:10097A0053656C65637420203E003C416D706C6960
:10098A00666963652056312E303E003C566F6C75A1
:10099A006D653A2020205B255D203E003C204465A1
:0E09AA006C617920446570746820203E000066
:00000001FF
